:100000000C9462000C947B1A0C94A81A0C948A002D
:100010000C948A000C948A000C948A000C948A0038
:100020000C948A000C948A000C948A000C948A0028
:100030000C948A000C94C2060C948A000C948A00DA
:100040000C94D51A0C948A000C94281E0C94631EF0
:100050000C948A000C948A000C948A000C948A00F8
:100060000C9446050C948A00000000002400270030
:100070002A0000000000250028002B0000000000DE
:1000800023002600290004040404040404040202DA
:100090000202020203030303030301020408102007
:1000A0004080010204081020010204081020000012
:1000B0000007000201000003040600000000000029
:1000C00000000B2011241FBECFEFD8E0DEBFCDBF54
:1000D00012E0A0E0B1E0ECE1F2E402C005900D9284
:1000E000A43CB107D9F714E0A4ECB2E001C01D9222
:1000F000AD3AB107E1F710E0C4ECD0E004C02297BC
:10010000FE010E940821C23CD107C9F70E9450207D
:100110000C940C210C940000FB01DC0102C0019046
:100120000D9241505040D8F708958091C40281301B
:1001300019F482E08093C4028091C402833019F4E0
:1001400084E08093C4020895E3E0F0E089E08093C6
:100150005700849190E08670863009F491E0892FF1
:1001600008951F93182F0E94A400882379F09FB749
:1001700081E08093F303F894A89588E18093600070
:1001800010936000112309F0A8959FBF1F91089557
:10019000382F20E08091F4039091F5038227932774
:1001A00040E061E270E19C01220F331F97FF04C021
:1001B000C9018627972701C0C9014F5F483099F7C9
:1001C0009093F5038093F40308958436910520F409
:1001D000BC0180E090E025C08E3B910550F48A552B
:1001E0009040BC0180E090E02AE030E040E050E048
:1001F00016C0823D910550F4845B9040BC0180E0C4
:1002000090E024E630E040E050E009C08D5C904092
:10021000BC0180E090E028E532E040E050E00E9440
:100220005F2024E630E040E050E00E945F20089527
:1002300090E08C599F4F0E94E5000895DC0198964C
:10024000EC91F0E0E770F070E455FD4F8081089587
:10025000FC0120A530E0C9018170907001962770E3
:10026000307035952795820F931F880F880F08955A
:100270008F929F92AF92BF92CF92DF92EF92FF92B6
:100280000F931F938C010E941E01D80197962C9109
:1002900030E043E150E0249FF001259FF00D349FB2
:1002A000F00D1124EC50FE4F80809180A280B3802D
:1002B00090E00F96AA2797FDA095BA2FBC01CD011B
:1002C00020E43FE14DE750E00E945F20A50194014A
:1002D0000E94922069017A0180ED97E0A0E0B0E0F1
:1002E000C80ED91EEA1EFB1ED80198968C91887103
:1002F00081F060E07EEE8AEB9BE0A50194010E9414
:10030000922028513C4F4F4F5F4FC20ED31EE41E28
:10031000F51E87EE93E0A0E0B0E0C80ED91EEA1EFD
:10032000FB1EC701B60128EE33E040E050E00E941A
:100330009220CA01B90128EE33E040E050E00E946B
:100340005F201F910F91FF90EF90DF90CF90BF90B3
:10035000AF909F908F9008951F93182FDB01FA01A3
:10036000482F469530E0848190E083709070982FFC
:1003700088272081820F911D11969C938E938481F2
:1003800090E08C70907076E0880F991F7A95E1F775
:100390002181820F911D13969C938E9312978481D5
:1003A00090E08073907064E0880F991F6A95E1F780
:1003B0002281820F911D15969C938E9314978481B0
:1003C00090E0807C9070880F991F880F991F23817F
:1003D000820F911D17969C938E93169735961896BB
:1003E0003F5F431708F0BFCF10FF50C08081829558
:1003F00086958695837090E02DE431E0AC01429FB4
:10040000C001439F900D529F900D11240C961196A0
:100410009C938E93808190E044E0969587954A95D1
:10042000E1F783709070AC01429FC001439F900D33
:10043000529F900D11240C9613969C938E931297B5
:10044000808190E0969587959695879583709070BA
:10045000AC01429FC001439F900D529F900D11240B
:100460000C9615969C938E931497808190E08370E0
:100470009070AC01429FC001439F900D529F900D20
:1004800011240C9617969C938E9316971F9108959E
:1004900023E08032920718F420E030E026C023E009
:1004A000883E920748F49C012F51334054E0369522
:1004B00027955A95E1F719C027E0803D920720F46F
:1004C0009C012C5D334011C028E08839920718F058
:1004D0002FEF33E00AC09C01285C374044E036959A
:1004E00027954A95E1F72D503C4FC90108958C306E
:1004F000910548F49C0174E0220F331F7A95E1F7CF
:10050000285D3C4F17C023E0843F920720F49C01F4
:1005100024523C4F0FC024E08030920718F020E9AD
:1005200038E008C09C012657334F64E0220F331F88
:100530006A95E1F7C90108959C01369527952575BF
:100540003575821B930B9C0136952795369527951B
:100550002373337383739373280F391FC901E4E046
:1005600096958795EA95E1F7820F931F8F709F709C
:1005700021E031E0AC01429FC001439F900D529FAA
:10058000900D1124892F0895882339F02D980000AB
:100590002B9A00002D9A000008952D9800002B98AA
:1005A00000002D9A000008952D9A000083B12D9827
:1005B000000090E0B4E096958795BA95E1F78170D8
:1005C00008950F931F93082F5C9A2D985C9810E064
:1005D000802F80780E94C402000F1F5F1830C1F77F
:1005E0002D981F910F9108958F770E94E102089531
:1005F0000F931F93082F10E0802F80780E94C40271
:10060000000F1F5F1830C1F72D981F910F910895AB
:100610000F931F932D9880E000E0182F110F0E9478
:10062000D402810F0F5F0830C1F71F910F91089519
:100630000E94F4020E9408035C9A08951F93162FEB
:1006400080680E94E102812F0E94F8025C9A1F914B
:1006500008951F931091E9021827E0EEF2E0E80FE9
:10066000F11D89E767850E941E038DE3612F0E94BB
:100670001E0382E4612F0E941E031F91089586E2EB
:100680000E94180308950F931F938BE20E94180392
:10069000082F8CE20E941803282F30E096E0369550
:1006A00027959A95E1F710E0000F111F000F111F19
:1006B000202B312BC9011F910F9108950F931F9388
:1006C0008C018CE1F80164810E941E038DE1F80128
:1006D00065810E941E038EE1F80166810E941E035F
:1006E00080E2F80167810E941E0381E2F8016085C3
:1006F0000E941E0382E2F80161850E941E0383E2CC
:10070000F80162850E941E0384E2F80163850E945D
:100710001E0385E2F80164850E941E038AE2F80147
:1007200065850E941E038EE6F80166850E941E0301
:100730008FE6F80167850E941E0380E7F801608953
:100740000E941E0381E7F80161890E941E0382E76F
:10075000F80162890E941E031F910F910895EF9284
:10076000FF920F931F93CF93DF937B018C01603037
:1007700028E372072CE982072CE1920728F520E88C
:1007800036E948E950E00E949220E9016897B901F2
:1007900080E090E020E839E647E65FEF0E945F20C6
:1007A0006E0D7F1D801F911F32E0660F771F881F1F
:1007B000991F3A95D1F721E732E040E050E00E94DE
:1007C0009220890180E421C020E03DE241E351E034
:1007D0000E949220E9016897B90180E090E020E052
:1007E00033ED4EEC5EEF0E945F206E0D7F1D801F8B
:1007F000911F660F771F881F991F21E732E040E0A5
:1008000050E00E949220890180E69E012F71622FA4
:10081000680F85E70E941E0386E7612F0E941E0372
:1008200087E7602F0E941E03CDB7DEB7E6E00C9489
:10083000F7209F92AF92BF92CF92DF920F93DF93F8
:10084000CF9300D000D0CDB7DEB7982E83E00E94C2
:1008500018038093090384E00E94180380930A031D
:1008600086E060E00E941E0387E061E00E941E03B4
:1008700089E06FE70E941E038AE065E00E941E0384
:100880008BE062E10E941E038CE065E10E941E0382
:100890008DE06DEF0E941E038EE060E00E941E035B
:1008A000992019F083E592E008C08091070323E1C5
:1008B000829FC00111248C509E4F0E945E0380E3F2
:1008C0006CE80E941E0382E36FE00E941E0383E334
:1008D00062E40E941E0384E36AE00E941E0385E333
:1008E0006AE20E941E0386E36DE20E941E0387E314
:1008F00064ED0E941E0388E360E00E941E0389E30A
:1009000060E00E941E03992049F065E8A62E61EC84
:10091000B62E61ECC62E6EEDD62E08C0A090E90270
:10092000B090EA02C090EB02D090EC020AE38D2D69
:100930009927AA27BB2789839A83AB83BC83802FFF
:1009400069810E941E03802F8B5F69810E941E03B4
:10095000DC2CCB2CBA2CAA240F5F0E3341F783E496
:100960006FEF0E941E0384E46FEF0E941E0385E474
:100970006FEF0E941E0386E46FEF0E941E03992012
:1009800019F08DE666E003C08DE66091ED020E94ED
:100990001E0389E760E00E941E038AE76091EE0271
:1009A0000E941E0383E760E00E941E0384E760E06C
:1009B0000E941E03992029F060EC7AEC89E896E306
:1009C00008C06091E5027091E6028091E702909183
:1009D000E8020E94AF030F900F900F900F90CF91FD
:1009E000DF910F91DF90CF90BF90AF909F900895CF
:1009F00087E061E00E941E038EE764E20E941E030E
:100A000088E063E00E941E0388E060E00E941E030D
:100A100087E065E00E941E0385E062E00E941E03FD
:100A200083E00E9418038093090384E00E94180366
:100A300080930A03089590E0411191E0880F982B6C
:100A40009093BA00660F6093BD003093100320931B
:100A50000F030895882311F085EC01C085E8809389
:100A6000BC00089585ED8093BC008091BC0084FD9E
:100A7000FCCF089585EC8093BC000895ECEBF0E08A
:100A8000108285E480831092150308951F920F92BF
:100A90000FB60F9211242F933F934F935F936F9351
:100AA0007F938F939F93AF93BF93EF93FF93DF93C6
:100AB000CF930F92CDB7DEB78091B90090E0887FD9
:100AC00090708036910509F4EAC081369105CCF525
:100AD0008832910509F47CC089329105B4F48031E3
:100AE000910509F470C0813191053CF4009709F437
:100AF0000EC1089709F00DC166C08831910509F44F
:100B000067C0809709F005C177C08034910509F46A
:100B100090C08134910544F48033910509F46EC08E
:100B2000C89709F0F6C06CC08035910509F471C012
:100B30008835910509F483C08834910509F0E9C02E
:100B4000A5C08839910509F4DCC089399105ECF418
:100B50008837910509F4A3C0893791054CF488368C
:100B6000910509F49CC08037910509F0D2C097C067
:100B70008838910509F4C5C08039910509F492C0FF
:100B80008038910509F0C5C08DC0803B910509F4FE
:100B9000A5C0813B91054CF4803A910509F499C0B8
:100BA000883A910509F0B5C099C0803C910509F4D7
:100BB000AAC0883C910509F4A6C0883B910509F0BC
:100BC000A8C080E08CC0809111038093BB009BC0C3
:100BD000809114038150809314038F5F09F43FC008
:100BE000E0911203F091130381918093BB00F09385
:100BF0001303E093120387C082E049C083E047C03B
:100C000084E080931603809115038B7F80931503F6
:100C100062C08091BB00E0911203F09113038193B5
:100C2000F0931303E0931203809114038150809397
:100C3000140380911403823008F065C062C0809173
:100C4000BB00E0911203F09113038193F09313031F
:100C5000E0931203809114038150809314038091D8
:100C600015038B7F809315038091150380FF4FC080
:100C7000809115038E7F8093150380911503826008
:100C80008093150384EA8093BC0043C085E0809381
:100C90001603809115038B7F8093150338C0109243
:100CA000140331C0E0910F03F0911003309749F124
:100CB0009091BB00809114038F5F80931403815047
:100CC00011F060E001C062E09983CE0101960995C0
:100CD0001BC00E9432050E943A051BC081E0E091D2
:100CE0000F03F0911003309761F0882311F461E055
:100CF00001C063E0CE010196099599819093BB00F4
:100D000003C080E001C081E00E942A0502C00E9469
:100D100032050F90CF91DF91FF91EF91BF91AF918D
:100D20009F918F917F916F915F914F913F912F9103
:100D30000F900FBE0F901F90189525B190E0FC0109
:100D4000EE0FFF1FE80FF91FE558FC4F8081282B9D
:100D500025B988B19181892B88B98BB19281892B72
:100D60008BB9089585B19091AB03892385B988B17A
:100D70009091AC03892388B98BB19091AD038923FD
:100D80008BB908951F920F920FB60F9211241F93E3
:100D90002F933F934F935F936F937F938F939F9383
:100DA000AF93BF93CF93DF93EF93FF9310914E03D5
:100DB00080918A02C0918802D0918902181708F0A8
:100DC0005BC08091AE039091AF03909387008093B6
:100DD0008600E12FF0E0EE0FFF1FEA59FD4F808102
:100DE00091810E947702880F991F9093AF0380939F
:100DF000AE038091AE039091AF039E01281B390B87
:100E0000C90130938902209388022091DB0230913E
:100E1000DC02220F331F8217930720F430938902DC
:100E20002093880280915003882339F48091D30263
:100E300080FF59C0183008F456C08FEF9FEF909391
:100E4000890080938800809184009091850080972C
:100E5000D0F30E94B20680914F03882339F4809129
:100E60004E03882319F081500E949D0680914E0305
:100E70008F5F80934E033EC08091AE039091AF038D
:100E80009093870080938600D093AF03C093AE0306
:100E900080915003882319F08FEF9FEF06C0809157
:100EA000AE039091AF038855924090938900809350
:100EB000880080E49CE99093890280938802809165
:100EC0008400909185008097D0F30E94B2068091B3
:100ED0004F03882329F480918A0281500E949D0645
:100EE00010924E0307C08091AE039091AF038855D6
:100EF0009240A5CFFF91EF91DF91CF91BF91AF913C
:100F00009F918F917F916F915F914F913F912F9121
:100F10001F910F900FBE0F901F90189590E0880FB3
:100F2000991F880F991F8C30910518F42CE030E040
:100F300007C09C0183E0253F380710F024EF33E021
:100F4000C901089580915203909153038F5F9F4F81
:100F5000E9F08091D402482F50E0A2E5B3E020E010
:100F600030E02417350761F0F8948D919C9111972A
:100F7000F901EE0FFF1FEA59FD4F918380837894AA
:100F80002F5F3F4F12962031310559F708951F9377
:100F9000CF93DF93EC0170E0CB018270907060FF23
:100FA0001AC0892B31F08091740388831092F20368
:100FB00045C01091F20380EE92E00E941E011817C6
:100FC000D8F5E12FF0E0E055FC4F808188831F5F6A
:100FD0001093F20333C0892BC1F098819093F103F1
:100FE0001092F203892F807E803651F48091740331
:100FF000823010F188818F718093330383E01AC0AF
:101000009E3FE1F41092740317C08091F1038F3F6B
:10101000A9F42091F203293278F4E22FF0E0E052B3
:10102000FD4F88818083822F8F5F8093F203893206
:1010300029F481E08093740380E001C081E0DF91B6
:10104000CF911F910895EF92FF920F931F93CF932B
:10105000DF9380E260E040E027EC37E00E941B0570
:1010600010927403E2E0EE2E75E0F72E04E080911A
:101070007403813039F480E00E941904E092740313
:101080005E98F5CF10917403133061F45D988091F0
:1010900033030E9429031093C4020E94F8040093B2
:1010A0007403E5CF80917403843009F78091C40202
:1010B0008430E9F68FE70E94F402C0E0D0E007C078
:1010C0000E940803FE01E055FC4F8083219680EECC
:1010D00092E00E941E0190E0C817D9078CF3F092AD
:1010E00074035D9AC4CFA0E0B0E0E9E7F8E00C94A7
:1010F000D720EC010E942B1B5B016C017E0100E0FC
:1011000010E011C0209779F00E942B1B6A197B090F
:101110008C099D09E616F7060807190720F40E94B6
:101120003E0581E008C08091150382FDEBCF8091E0
:10113000160310921603CDB7DEB7EAE00C94F32045
:10114000A0E0B0E0E6EAF8E00C94D920182F7B018B
:10115000042FC22FD0E0F4E0CF2ED12CCC22DD2200
:1011600022FF03C080E090E004C08091860290914D
:1011700087020E947308282F8823B9F5109216035E
:1011800000931403F0921303E0921203110F116005
:101190001093110390911503C1FD02C084E001C0BA
:1011A00085E0892B809315038091150381FF0BC087
:1011B000809115038D7F8093150380911103809397
:1011C000BB0085EC01C085EE8093BC00C0FF0DC064
:1011D000C114D10419F080E090E004C0809186022F
:1011E000909187020E947308282F822FCDB7DEB717
:1011F000E8E00C94F520A0E0B0E0E1E0F9E00C9428
:10120000D920182F7B01042FC22FD0E0A4E0CA2ED2
:10121000D12CCC22DD2222FF03C080E090E004C06C
:1012200080918602909187020E947308282F88235C
:10123000B1F51092160300931403F0921303E09299
:101240001203110F1093110390911503C1FD02C0F9
:1012500084E001C085E0892B8093150380911503FC
:1012600081FF0BC0809115038D7F809315038091C2
:1012700011038093BB0085EC01C085EE8093BC0018
:10128000C0FF0DC0C114D10419F080E090E004C08B
:1012900080918602909187020E947308282F822FE6
:1012A000CDB7DEB7E8E00C94F5208091C402813020
:1012B00011F081E008950E942B1B20910B033091C7
:1012C0000C0340910D0350910E03621B730B840BB2
:1012D000950B615A76488140904010F480E0089563
:1012E00082E00895FF920F931F93CF93DF93182FFF
:1012F000092FF62E8EE30E941E03212F302FC901E5
:10130000EC0110E005C08FE769910E941E031F5F8A
:101310001F15C8F385E064E00E941E0383E00E946D
:1013200018038093090384E00E94180380930A0342
:101330000E942B1B60930B0370930C0380930D038F
:1013400090930E0387E069E00E941E0381E0809382
:10135000C402CDB7DEB7E5E00C94F8200E94720914
:101360008091C4028130D9F40E942B1B20910B0381
:1013700030910C0340910D0350910E03621B730BCF
:10138000840B950B605A76488140904040F4E8CF3A
:101390008BE894E060E071E00E94131E0895809154
:1013A000C4028130A9F30895A1E0B0E0EAEDF9E0CC
:1013B0000C94DF20809174038230B9F480E2BE0186
:1013C0006F5F7F4F41E021E00E94A008882379F001
:1013D0008FEF809374030E941D1B609375037093BD
:1013E000760380937703909378038FEF01C0898110
:1013F0002196E2E00C94FB20A1E0B0E0E2E0FAE00C
:101400000C94DF20809174038230D9F480913303EF
:10141000805A898380E2BE016F5F7F4F41E021E007
:101420000E94FB08882369F08FEF809374030E9469
:101430001D1B6093750370937603809377039093DD
:1014400078032196E2E00C94FB20AAE2B0E0EBE204
:10145000FAE00C94DD208FEF8983DE011296E0EE36
:10146000F2E089E201900D928150E1F780E28E0175
:101470000F5F1F4FB8014AE221E00E94FB0888235A
:1014800051F480E2B80141E021E00E94A0088823E5
:1014900011F482E001C08FEF809374038091740394
:1014A000823051F00E941D1B609375037093760388
:1014B0008093770390937803AA96E4E00C94F92044
:1014C000A2E0B0E0E6E6FAE00C94DB200E942B1BE1
:1014D0009B01AC018091170390911803A09119030F
:1014E000B0911A0379018A01E81AF90A0A0B1B0B59
:1014F000D801C70181519742A040B04008F444C0D0
:1015000080911B038F5F80931B03815080FD02C07D
:1015100000E001C007E020931703309318034093C5
:10152000190350931A038BE894E063E00E94CB1FE9
:101530008BE894E061E00E94CB1F47E0F42EF00EB0
:10154000802F90E0880F991F9C012A593D4F3A83C4
:101550002983F90160817181672F7727637070702B
:10156000880F991F682B792B8BE894E00E94CB1F82
:10157000E981FA816081718170708BE894E00E944A
:10158000CB1F0F5F0F15E1F62296E6E00C94F720D3
:101590001F93182F8BE894E0612F0E94CB1F812F9F
:1015A0000E94C8001F910895A0E0B0E0EAEDFAE0C3
:1015B0000C94D920082F0E942B1B9B01AC01809119
:1015C000170390911803A0911903B0911A036901B0
:1015D0007A01C81AD90AEA0AFB0AD701C601815161
:1015E0009742A040B04008F443C0209317033093C3
:1015F00018034093190350931A031092F5031092A5
:10160000F40388EA0E94C80A002311F481E001C0B3
:1016100081E80E94C80A80E10E94C80AC0E0D0E0C8
:10162000FE01EE0FFF1FEA59FD4F808191810E945C
:1016300077028C0153E0000F111F5A95E1F7812FBB
:101640000E94C80A802F0E94C80A2196C031D10585
:1016500039F76091F5038BE894E00E94CB1F60910D
:10166000F4037091F50370708BE894E00E94CB1F37
:10167000CDB7DEB7E8E00C94F520A0E0B0E0E3E4FD
:10168000FBE00C94D920182F062F0E942B1B9B01E6
:10169000AC018091170390911803A0911903B091A8
:1016A0001A0369017A01C81AD90AEA0AFB0AD701A2
:1016B000C60181519742A040B04008F4D6C12093A2
:1016C0001703309318034093190350931A03809122
:1016D000660290916702880F991F80931C03977090
:1016E00080911D03887F892B80931D0320916802C0
:1016F00030916902220F331F922F990F990F990F82
:101700008770892B80931D03422F42954695477021
:1017100080911E03807C932F9770990F990F990FDA
:10172000842B892B80931E0320916A0230916B02D7
:10173000220F331F922F9295990F990F907C8F73E0
:10174000892B80931E03932F9295990F990F907C6C
:10175000822F86958695892B80931F03932F9695CC
:1017600096959170809120038E7F892B8093200322
:1017700020916C0230916D02220F331F922F990F2E
:101780008170892B80932003422F441F4427441FDC
:1017900080912103807F932F9770990F842B892B41
:1017A0008093210320916E0230916F02220F331F2C
:1017B000922F9295907F8F70892B80932103422FD7
:1017C00042954F70809122038078932F9770929565
:1017D000907F842B892B809322032091700230917B
:1017E0007102220F331F8F7780932203932F9795D7
:1017F00099279795822F8695892B80932303932F82
:1018000096959370809124038C7F892B8093240379
:101810004091720250917302440F551F942F990FFB
:10182000990F8370892B80932403942F929596951A
:101830009695937020912503207E852F8770880FC1
:10184000880F292B282B20932503809174029091D7
:101850007502880F991F382F3295330F307E2F7104
:10186000232B20932503292F2295220F207E869556
:1018700086958695822B809326038091760290919F
:101880007702880F991F8093270397708091280310
:10189000887F892B809328032091780230917902E8
:1018A000220F331F922F990F990F990F8770892B51
:1018B00080932803422F42954695477080912903D3
:1018C000807C932F9770990F990F990F842B892BF8
:1018D0008093290320917A0230917B02220F331FDB
:1018E000922F9295990F990F907C8F73892B8093EB
:1018F0002903932F9295990F990F907C822F8695AB
:101900008695892B80932A03932F969596959170AF
:1019100080912B038E7F892B80932B0320917C0257
:1019200030917D02220F331F922F990F8170892BE6
:1019300080932B03422F441F4427441F80912C0384
:10194000807F932F9770990F842B892B80932C0382
:1019500020917E0230917F02220F331F922F9295A9
:10196000907F8F70892B80932C03422F42954F706C
:1019700080912D038078932F97709295907F842B80
:10198000892B80932D032091800230918102220FB8
:10199000331F8F7780932D03932F979599279795D2
:1019A000822F8695892B80932E03932F9695937083
:1019B00080912F038C7F892B80932F03409182028B
:1019C00050918302440F551F942F990F990F8370E4
:1019D000892B80932F03942F9295969596959370CB
:1019E00020913003207E852F8770880F880F292B48
:1019F000282B209330038091840290918502880FD8
:101A0000991F382F3295330F307E2F71232B20935F
:101A10003003292F2295220F207E86958695869564
:101A2000822B80933103112311F490E001C098E0E0
:101A3000002311F480E001C084E0892B80933203FD
:101A40008BE894E06FE00E94CB1FCCE1D3E08BE801
:101A500094E069910E94CB1F83E0C333D807B9F7A4
:101A60008BE894E060E00E94CB1FCDB7DEB7E8E0E2
:101A70000C94F5201F93182F8091CB028B3221F408
:101A80008FE0612F0E94261C8091C802873259F492
:101A9000112321F08091B000806103C08091B000DB
:101AA0008F7E8093B0001F9108950F931F938091B4
:101AB0004C0390914D039F770E949C02982F8F308A
:101AC00029F4809148038695805804C089E0989F46
:101AD000C0011124809349030091D402003170F4B5
:101AE000F89410E0809149030E948E07000F111FA7
:101AF0000A591D4FF8019183808378948091C80220
:101B00008132C9F490914903892F81508E3F60F052
:101B10008091B0008F7D8093B00060E0911161E012
:101B200083E00E94261C07C09093B4008091B0000F
:101B300080628093B0001F910F9108951F93182F1A
:101B4000811111E082E1612F0E94261C83E1612F47
:101B50000E94261C10921403109215038091B90064
:101B60008C6F8093B90080E28093B80085E4809305
:101B7000BC001F910895CF93DF938BE894E00E94FF
:101B8000581F892BF9F08091EF03C82FD0E09E01F8
:101B90002F5F3F4F2F7130708091EE0390E0281738
:101BA000390781F08BE894E00E94921FC253DC4F0A
:101BB00088838091EF0390E001968F7190708093FD
:101BC000EF03DBCFDF91CF910895EF92FF921F9348
:101BD000CF93DF9380EE92E00E94280180938A02E7
:101BE0009091D402981719F49F5F90938A02EBE7C3
:101BF000F3E0108211821282339623E0E339F20778
:101C0000C1F78FEF8093AB038093AC038093AD0358
:101C1000E6ECEE2EE2E0FE2EA4E9B2E0E7016FEF83
:101C20005FEF4FEF88818031F0F490E03C91FC0150
:101C3000EE0FFF1FE80FF91FE558FC4F8081832B43
:101C4000808311962C9111978181822B818312962A
:101C50009C9112978281892B828330954323209512
:101C60005223909569232196139682E0CE3CD807A3
:101C7000C9F66093AD035093AC034093AB03CCE83B
:101C8000D2E010E0F7018081823238F08632B0F085
:101C9000863219F4888160E00FC0163021F48091FB
:101CA000C1008F7E05C0173029F48091C100877F65
:101CB0008093C100888161E00E94BA1B1F5F089475
:101CC000E11CF11C21961830E9F68091C6028032A1
:101CD00031F489E061E00E94261C82E801C082E0C4
:101CE0008093800081E080934F0380935003809124
:101CF000C802813211F08732C9F483E061E00E94AA
:101D0000BA1B83E060E00E94261C8091C8028132E9
:101D100021F481E08093B00009C082E08093B0009C
:101D200085E08093B1008EE38093B3008AE18093D5
:101D300081008FEF9FEF909389008093880080ED62
:101D400097E0909387008093860080E49CE99093CD
:101D50008902809388029093AF038093AE03109220
:101D60004E0380916F00816080936F008091D30259
:101D700083FF0DC080915203909153038F5F9F4F5B
:101D800031F00E94A2071092500310924F03DF918E
:101D9000CF911F91FF90EF9008958CE060E00E943A
:101DA000BA1B8BE061E00E94BA1B8DE061E00E94EB
:101DB000BA1B82E060E00E94BA1B84E061E00E94EE
:101DC000BA1B089583E00E9418038093090384E0FE
:101DD0000E94180380930A0387E061E00E941E03BB
:101DE0006AE070E080E090E00E94511B0E94F804DD
:101DF000000008950F931F93082F17C05E9A64E6A2
:101E000070E080E090E00E94511B5E9864E670E014
:101E100080E090E00E94511B1F5F101778F36CE286
:101E200071E080E090E00E94511B10E0F6CF482F57
:101E3000392F25E00DC0F999FECF1FBA842F932FBB
:101E400092BD81BD60BD0FB6F894FA9AF99A0FBEA3
:101E5000215059F0F999FECF842F932F92BD81BD67
:101E6000F89A80B5681739F7089582E00E94FA0E53
:101E70000895A0E0B0E0EFE3FFE00C94D120482EFD
:101E8000562EEE24FF24C0E0D0E0CC24DD248824AC
:101E9000992404C055245394CC24DD24442051F4C7
:101EA00085ECE82E82E0F82EC0E0D0E00BE1802E39
:101EB000912C19C021E0421651F410EEE12E12E0EF
:101EC000F12ECDE1D0E0B9E28B2E912C0CC032E0A6
:101ED000431649F4A2E5EA2EA3E0FA2EC8E4D0E0C6
:101EE000F0E28F2E912C3E016C0C7D1C1092F503BC
:101EF0001092F403E3011BC0552059F4F999FECF69
:101F0000D2BDC1BDF89A80B5F701E00FF11F808303
:101F100007C0F701E00FF11FCE0160810E94170F8B
:101F20000E0D1F1DF80180810E94C80021969E01A0
:101F30002619022F10E008151905F0F2CE015520E0
:101F4000D9F4F999FECFD2BDC1BDF89A20B5F9995F
:101F5000FECF2196D2BDC1BD2197F89A80B590E001
:101F6000B22EAA248A299B292091F4033091F503EB
:101F70002817390759F48ECF21966091F5030E94F6
:101F8000170FCE016091F4030E94170F80E091E0DB
:101F9000C80ED91E91E0C91693E0D90608F47ECF89
:101FA000852DCDB7DEB7E0E10C94ED2082E060E056
:101FB0000E94390F882331F48FEF9FEF90935303E2
:101FC00080935203089582E061E00E94390F0895E2
:101FD00095E09093C50290E29093C60292E29093AE
:101FE000C70291E29093C80293E29093C9029BE2E8
:101FF0009093CB0294E29093CC0295E29093CD0221
:1020000092E09093D3029FEF9093D4022AE0209322
:10201000DD021092DE021092DF021092D5021092C1
:10202000D6021092D7021092D8029EE19093D90264
:102030002093DA0228EB3BE03093DC022093DB02B2
:10204000882361F080E061E00E94390F8FEF9FEFFD
:1020500090935303809352030E94E30F0895A3E6E5
:10206000B0E0E5E3F0E10C94CF205B016C010E944D
:102070001D1B1B012C0181E00E94190483E0809349
:10208000C4020E94E20E8BE894E06CE071E00E94D2
:10209000131E3E010894611C711C2FE330E02C0FCD
:1020A0003D1F2B5F3F4FA4963FAF2EAFA497EEC0CE
:1020B0008BE894E06AE171E00E94131E8FE70E94B2
:1020C000F4020E940803182F8983823601F500EE7E
:1020D00012E00E940803F80181938F01F3E00930B8
:1020E0001F07B9F78091E002873309F0CAC08BE877
:1020F00094E063E271E00E94131E82E48983CE01C2
:10210000019661E00E94AE095D9A81E0D5C08037FA
:1021100019F0893631F506C020E52A83AA24BB24AC
:10212000650105C081E00E94E80F89E48A838091FF
:10213000F303882321F08091D302806803C080914B
:10214000D3028F778093D302DE011396E5ECF2E0A1
:102150008BE101900D928150E1F7CE0102966CE186
:102160008EC0843731F584E58FAF33E021963FAFE1
:10217000219780E722968FAF229788E023968FAF32
:1021800023978FE024968FAF2497A496AEADBFAD72
:10219000A497E6EDF1E08EE101900D928150E1F718
:1021A000CE01CF9663E20E94AE09AA24BB2465014A
:1021B00068C0853791F405EC12E00E940803F8012D
:1021C00081938F01F2E0003E1F07B9F780E061E0E4
:1021D0000E94390F25E5298350C0863631F580915C
:1021E0005203909153038F5F9F4FD1F086E48E8FFF
:1021F00092E5E92E93E0F92E8E01015E1F4FF70163
:10220000819191917F010E947702F80190838183EF
:102210000E5F1F4FF2E7EF16F3E0FF0681F701C0F4
:102220001E8FCE014E9661E22AC08736D9F402E5B0
:1022300013E00E940803982E88240E94080394014A
:10224000280F311DC9010E944802F8018193919322
:102250008F01F3E002371F0761F727E429830E940B
:10226000E30F0BC0873469F48FEF9FEF9093530314
:10227000809352030E94E30F1983C30161E00E941F
:10228000AE0993E09093C4020E94F804A114B10433
:10229000C104D10459F00E941D1B621973098409FD
:1022A00095096A157B058C059D0528F48091C4026B
:1022B000843061F7FDCE80E0CD59DF4FE2E10C9430
:1022C000EB2080E060E00E94390F882319F481E060
:1022D0000E94E80F089581E061E00E94390F08959F
:1022E00081E060E00E94390F882311F490E006C07D
:1022F00090E08091E002873309F491E0892F0895FE
:10230000EF92FF920F931F93CF93DF93EB019C010A
:10231000442737FD4095542F60E271EA87E090E052
:102320000E94B42089011216130614F001E010E097
:10233000BE01882777FD8095982F20E231EA47E09B
:1023400050E00E945F209801442737FD4095542FAC
:102350000E94B4207901C0E0D0E009C02B9AC801E6
:102360000E94751B2B98C8010E94751B2196CE15E3
:10237000DF05A4F3CDB7DEB7E6E00C94F7205D9A55
:1023800083E00E9418038093090384E00E941803ED
:1023900080930A0386E060E00E941E0387E061E00C
:1023A0000E941E0389E06FE70E941E038AE065E039
:1023B0000E941E038BE062E10E941E038CE065E137
:1023C0000E941E038DE06DEF0E941E038EE060E010
:1023D0000E941E0380E76CE20E941E0380E360E01F
:1023E0000E941E0389E760E00E941E038AE765E001
:1023F0000E941E0381E762E10E941E0382E762E001
:102400000E941E0383E760E00E941E0384E760E0F1
:102410000E941E036091D5027091D6028091D7026E
:102420009091D8020E94AF038DE667E00E941E03E0
:102430006AE070E080E090E00E94511B87E069E074
:102440000E941E036AE070E080E090E00E94511B51
:1024500088E891E061E070E00E948011A8958DE627
:1024600065E00E941E036AE070E080E090E00E9458
:10247000511B88EB91E061E070E00E948011A8950B
:102480008DE664E00E941E036AE070E080E090E068
:102490000E94511B8DE591E061E070E00E94801187
:1024A000A8958DE662E00E941E036AE070E080E07D
:1024B00090E00E94511B8FEA90E061E070E00E9482
:1024C0008011A8958DE660E00E941E036AE070E02E
:1024D00080E090E00E94511B85E091E062E070E0B6
:1024E0000E948011A89587E061E00E941E035D981C
:1024F0000895A6E1B0E0EFE7F2E10C94D120A895B1
:102500008CE00E941803882359F48BE894E06EE273
:1025100071E00E94131E80E00E9419040E94E20EE6
:102520000E94BB0D0E942B1B0E94D409B82E8E0165
:102530000F5F1F4FAA24AA948091C402843029F00F
:1025400045E0E42EBE1409F0A2C10E942B1B6B01D2
:102550007C018091C4028430E9F48FE70E94F40288
:1025600000E010E008C00E940803F801E055FC4FAD
:1025700080830F5F1F4F80EE92E00E941E0190E06B
:102580000817190784F30E94430390934B03809329
:102590004A0328C080EE92E00E941E01482F4F5F40
:1025A00080E2B80121E00E94A008882369F0A0928F
:1025B00074030E941D1B60937503709376038093D0
:1025C000770390937803B8CF80EE92E00E941E01CB
:1025D000482F20EB33E0FE013296C901BF0150E0E5
:1025E0000E948C00C0923403D0923503E0923603EF
:1025F000F09237031092730380914C0390914D0336
:10260000880F991F816090934D0380934C035E98CF
:102610005D9A80E00E943A0D8091B003282F30E04F
:10262000C9018E739070892B09F041C0F894809194
:102630000803877066E672E041EB53E00E94AC014C
:102640000091D402003160F410E0809149030E94AF
:102650008E07000F111F0A591D4FF80191838083C7
:1026600078948091B00390917A0380FF1BC09923E6
:1026700009F045C0A2E5B3E020E030E0F901EE0F3B
:10268000FF1FEA59FD4F808191818D939D932F5FAC
:102690003F4F2031310591F70E94E30F81E0809395
:1026A0007A032DC0992359F110927A0328C0C901E9
:1026B00088739070C89719F54091C503842F8227BD
:1026C00087FF1DC040584093C5038091CD028532DD
:1026D000B1F410E00AC01F5FE12FF0E0E055FC4FBD
:1026E0008BE894E060810E94CB1F212F30E0809125
:1026F000B00390E0877090708217930764F7809121
:102700007203882319F481E08093720310925103BD
:1027100010924F031092500380910803887109F4BE
:10272000ADC04091C5038091B00390E0242F30E00C
:102730008227932786FD6CC0407C80E44827409325
:10274000C5039091EE038091EF03981701F1A6EC79
:10275000B3E030E00FC03F5F892F90E0FC01E2530F
:10276000FC4F20812D9301968F7190708093EE0322
:10277000383031F09091EE038091EF03981759F7BC
:10278000395C8091C503382B3093C50341C08091DB
:1027900047038093C6038091C702863211F482E119
:1027A00005C08091CA02863251F48EE00E94891CD5
:1027B00095958795959587958093C70302C010924C
:1027C000C7038091C902863211F483E105C080916C
:1027D000CB02863251F48FE00E94891C9595879533
:1027E000959587958093C80302C01092C803809185
:1027F0004B038093C90380914A038093CA0380915D
:102800004C0390914D039F770E949C028093CB03D1
:1028100085EC93E069E00E94720902C00E94BB0D42
:102820000E9455098823D1F306EC12E05CE8E52EFE
:1028300052E0F52EF8018081E82FF0E0CF01807F93
:102840009070409791F4EF70F070EE0FFF1FEA590F
:10285000FD4F8081918160E08F3F910511F008F07C
:1028600061E0F70180810E94261C0F5F1F4F0894D2
:10287000E11CF11CF2E00E3C1F07E1F683E08093BF
:10288000C4020E94F80481E0809379035D980E945D
:102890002B1B5B016C010E941D1B2B013C018091D5
:1028A0007303823008F065C0E0903403F090350384
:1028B00000913603109137038091380390913903CA
:1028C000A0913A03B0913B038E159F05A007B10775
:1028D00009F44FC080EE92E00E943801A6019501F4
:1028E0002E193F09400B510B6C5D754080409040A4
:1028F0006217730784079507E0F5E0923803F092BA
:10290000390300933A0310933B030E943F038093E3
:1029100047032091450330914603280F311D309322
:10292000460320934503609144036F5F6093440323
:102930006930F8F0C90170E00E947E20CB017093ED
:102940004603609345032091480343E0249F900190
:102950001124820F931F969587959695879580935E
:1029600048030E94550D10924603109245031092A1
:102970004403809172039090F003882309F457C1B7
:1029800080907303891408F0D5C180EE92E00E9414
:102990003801209134033091350340913603509132
:1029A0003703A21AB30AC40AD50A68517C4F8F4F65
:1029B0009F4F6A157B058C059D0508F075C08091B9
:1029C0004C0390914D03880F991F90934D03809372
:1029D0004C0381E080937903882081F440923C038A
:1029E00050923D0360923E0370923F031092400369
:1029F000109241031092420310924303809173039B
:102A00008F5F8093730380EE92E00E9438012091E3
:102A10003403309135034091360350913703260F2C
:102A2000371F481F591F20933403309335034093B9
:102A300036035093370381E0809379035E9A0E94B6
:102A40003A0D0E94550D30C080EE92E00E94380190
:102A50009B01AC018091340390913503A091360322
:102A6000B091370386017501E81AF90A0A0B1B0BAE
:102A7000682D70E080E090E00E945F206E157F0579
:102A80008007910788F410924D0310924C0381E067
:102A9000809379030E94550DA0923403B0923503C0
:102AA000C0923603D092370380917303882309F4D0
:102AB000E8C09091DD02992389F180915103882328
:102AC00069F5892F90E00E94E50020913C03309148
:102AD0003D0340913E0350913F0383017201E21A8E
:102AE000F30A040B150B6E157F0580079107B0F4F0
:102AF00081E0809351030E94A2078091D9020E9435
:102B00001801640D751D861D971D6160609340035B
:102B10007093410380934203909343039091DF02AB
:102B20009923F1F080914F038823D1F4892F90E00D
:102B30000E94E50020913C0330913D0340913E030B
:102B400050913F0383017201E21AF30A040B150B43
:102B50006E157F058007910718F481E080934F037D
:102B60009091DE029923F1F0809150038823D1F4F3
:102B7000892F90E00E94E50020913C0330913D03B5
:102B800040913E0350913F0383017201E21AF30A20
:102B9000040B150B6E157F058007910718F481E073
:102BA000809350038091D5029091D602A091D702D4
:102BB000B091D8020097A105B10509F462C08091D7
:102BC000400390914103A0914203B09143030097C9
:102BD000A105B10509F455C083017201E81AF90A8B
:102BE0000A0B1B0B17FD4DC06091DA0270E080E00C
:102BF00090E028EE33E040E050E00E945F206E1548
:102C00007F0580079107E8F50E94BF1180E00E94D0
:102C100019040E94F8040E941D1B61606093400328
:102C20007093410380934203909343032AC080EE44
:102C300092E00E9438019B01AC0180913403909195
:102C40003503A0913603B091370386017501E81A68
:102C5000F90A0A0B1B0B692D70E080E090E00E94DE
:102C60005F206E157F058007910758F4A09234030A
:102C7000B0923503C0923603D092370381E080933F
:102C80007903809150038823B1F48091CD0288327A
:102C900019F40E94600A0FC0893239F480915103FF
:102CA000609173030E943D0B06C08A3221F480912B
:102CB00051030E94D40A809179038823B9F0E091EE
:102CC0003303EF5FE0933303E83131F0F0E0E0529B
:102CD000FD4F8785882311F41092330380913303CD
:102CE0000E9429030E94FC091092790380917403C9
:102CF0008F3F21F50E941D1B2091750330917603B3
:102D00004091770350917803621B730B840B950BF2
:102D1000695E73408040904088F00E941D1B609364
:102D200075037093760380937703909378030E94E2
:102D3000250A04C0891409F0B7CE86CE6696E0E174
:102D40000C94ED20FF920F931F93082FF62E61E055
:102D50000E94BA1B802F61E00E94261C8F2D61E02B
:102D60000E94261C8AE090E00E94751B8F2D0E9415
:102D7000591C892B11F410E00FC0802F60E00E94D5
:102D8000261C8AE090E00E94751B8F2D0E94591C22
:102D900010E0892B09F411E0802F60E00E94BA1B3B
:102DA000802F60E00E94261C8F2D60E00E94261C70
:102DB000812F1F910F91FF900895EF92FF920F9333
:102DC0001F938C016BE8E62E64E0F62EC701612F9D
:102DD00070E04AE050E00E94901DC7016EE20E9440
:102DE000CF1C54E0169507955A95E1F70F701070B7
:102DF000C701B8014AE050E00E94901D1F910F9159
:102E0000FF90EF900895A2E2B0E0E9E0F7E10C94C2
:102E1000CF208E010F5F1F4F80E1D8011D928A9550
:102E2000E9F78BE894E066E371E00E94131E0E94CC
:102E3000E20E20EC3DE948E555E32F8F38A349A386
:102E40005AA380EC97EFAAEBB7E38B8F9C8FAD8FE3
:102E5000BE8F24EF31E040E050E02F8B388F498F58
:102E60005A8FA0E5CA2EA3ECDA2EE12CF12CF0EC5F
:102E70004F2EFDE95F2EF8E56F2EF5E37F2E8824B7
:102E80009924540133241E8A1D8A198A1A8A1B8A9E
:102E90001C8AFFC08BE894E00E94921F8434B9F032
:102EA000853430F48332B9F18C3209F0CCC044C09F
:102EB000833509F0C8C02F8D38A149A15AA1C90195
:102EC000DA012C013D01882499245401E2C08BE8E9
:102ED00094E064E40E94CF1C8BE894E040EC5DE950
:102EE00068E575E32AE030E00E94B31D8BE894E0CA
:102EF0006CE20E94CF1C8BE894E040EC57EF6AEB49
:102F000077E32AE030E00E94B31D8BE894E06CE2A6
:102F10000E94ED1CBEC019821A821B821C821D8277
:102F20001E821F82188619861A861B861C861D869D
:102F30001E861F86188A3AC0339434E0331609F08F
:102F4000A8C069817A818B819C8128EE33E040E0C2
:102F500050E00E945F206F8F78A389A39AA36D81B0
:102F60007E818F8198850E945F206B8F7C8F8D8FF3
:102F70009E8F89859A85AB85BC858F8B988FA98F0D
:102F8000BA8F6D857E858F8598890E945F206B0141
:102F90007C0190E2C9169EE4D90690E0E90690E033
:102FA000F90630F48CE162E30E941E03332471C001
:102FB000A0E3CA16A5E7DA06A0E0EA06A0E0FA0652
:102FC00018F48CE162E2F0CFB0E4CB16BCE9DB068A
:102FD000B0E0EB06B0E0FB0618F48CE166E2E4CF6B
:102FE000E0E5CE16E3ECDE06E0E0EE06E0E0FE060D
:102FF00018F48CE162E1D8CFF0E6CF16FAEEDF06E6
:10300000F0E0EF06F0E0FF0618F48CE165E1CCCFCC
:1030100020E7C21621E1D20621E0E20620E0F20616
:1030200018F48CE161E0C0CF30EAC31636E8D3066D
:1030300031E0E30630E0F30618F48CE163E0B4CF4E
:103040008CE165E0B1CFE0ED2E2E280E49E042156F
:1030500000F1032D10E0000F111F000F111F81E080
:1030600090E08C0F9D1F080F191FD8016D917D9165
:103070008D919C912AE030E040E050E00E945F207A
:10308000620D711D811D911DF80160837183828322
:1030900093838BE894E00E94581F892B09F0FACEA5
:1030A00081149104A104B10489F4C301B2010E9406
:1030B000AF0361E070E080E090E00E94511BFFEF01
:1030C000FE8B1D8A198A1A8A1B8A1C8A2F89388DC1
:1030D000498D5A8D82169306A406B506E0F40E9427
:1030E0003F0329893A894B895C89280F311D411D8D
:1030F000511D298B3A8B4B8B5C8B3D89381708F41B
:103100008D8B4E89841708F48E8B0894811C911C3A
:10311000A11CB11C56C0C301B20128EE33E040E04F
:1031200050E00E9492208BE894E0BA01A9012AE0C5
:1031300030E00E94811D8BE894E06CE20E94CF1C7D
:103140008BE894E06D894AE050E00E94A11D8BE875
:1031500094E06CE20E94CF1C69897A898B899C89F2
:10316000A50194010E9492208BE894E0BA01A90184
:103170002AE030E00E94811D8BE894E06CE20E941E
:10318000CF1C8BE894E06E894AE050E00E94A11DBC
:103190008BE894E06CE20E94ED1C4C0C5D1C6E1CF4
:1031A0007F1C8B8D9C8DAD8DBE8D84159505A605E0
:1031B000B70520F44F8C58A069A07AA088249924E0
:1031C00054012F8D38A149A15AA1285E33404040B7
:1031D000504009F05ECFA296E2E10C94EB2080E033
:1031E00065E970E042E050E00E94581A0895A1E0BD
:1031F000B0E0EDEFF8E10C94DF2080E00E94B10038
:1032000085E061E00E94BA1B86E061E00E94BA1B83
:103210000E94CD0E80E060E00E94BA1B81E061E078
:103220000E94BA1B8BE894E040E052EC61E070E051
:103230000E94D11E0E9461110E94D60F8BE894E07B
:1032400063E471E00E94101E80E793E00E94DD16A7
:103250008BE894E06AE571E00E94101E8BE894E030
:1032600067E070E04AE050E00E94FC1D0E94EF1809
:1032700078945E9A83E063E10E94A216882329F085
:103280005E985D980E940317FBCF89E062E10E947F
:10329000A216882329F40E947011882309F000C126
:1032A0008BE894E062E671E00E94101E60E070E03E
:1032B00080E090E00E942F10882349F00E946B115B
:1032C0008BE894E06BE971E00E94131E5D9A0E9406
:1032D000E50D22C08091C902833229F08091D3028A
:1032E0008B7F8093D3028091D30281FF15C082FD32
:1032F00013C064EF71E080E090E00E942F108823FB
:1033000059F00E946B118BE894E06BE971E00E9428
:10331000131E0E94E50D5D9A8091C702823239F535
:103320008091C902833219F581E00E949E0D80913F
:10333000D30282FF09C08BE894E066EB71E00E9443
:10334000131E0E94230813C064E170E080E090E047
:103350000E94511B80E2BE016F5F7F4F41E021E080
:103360000E94A008882319F481E0809374038BE8FD
:1033700094E061EC71E00E94101E8FE00E94B100A9
:1033800080E00E9419041092330380E00E94290318
:103390001092F00390E0983158F4292F2F5FE92F15
:1033A000F0E0E052FD4F8785882311F0922FF3CF94
:1033B0009093F00383E08093C4020E94E20E809118
:1033C0007403882311F00E94250A8091CD0288326F
:1033D00011F08A3239F48BE894E040E052EC61E07D
:1033E00070E02BC0893271F48BE894E040EA56E833
:1033F00061E070E00E94D11E8091C20080628093E3
:10340000C20022C0809108038871803169F0409128
:10341000E1025091E2026091E3027091E4024A30CD
:1034200051056105710538F48BE894E040E855E2F8
:1034300060E070E002C08BE894E00E94D11E04C0FE
:103440008BE894E00E94921F8BE894E00E94581F42
:10345000892BB1F78091CC02843229F08091C10090
:103460008F7E8093C1008091CD02853229F08091BA
:10347000C100877F8093C1001092EE031092EF038A
:10348000109272030E942B1B6093340370933503D8
:1034900080933603909337032196E2E00C94FB204F
:1034A0000E94E50D8091C702823209F017CF12CF3A
:1034B000823000F5E82FF0E0EE0FFF1FEA50FC4FDE
:1034C00071836083882319F08130A1F408C0809152
:1034D00069008C7F842B80936900E89A089580911D
:1034E0006900440F551F440F551F837F842B809321
:1034F0006900E99A08951F920F920FB60F92112456
:103500002F933F934F935F936F937F938F939F93EB
:10351000AF93BF93EF93FF938091F6039091F703DE
:10352000892B29F0E091F603F091F7030995FF91BB
:10353000EF91BF91AF919F918F917F916F915F912B
:103540004F913F912F910F900FBE0F901F901895A4
:103550001F920F920FB60F9211242F933F934F9308
:103560005F936F937F938F939F93AF93BF93EF93EB
:10357000FF938091F8039091F903892B29F0E09152
:10358000F803F091F9030995FF91EF91BF91AF9185
:103590009F918F917F916F915F914F913F912F916B
:1035A0000F900FBE0F901F9018951F920F920FB69D
:1035B0000F9211242F933F938F939F93AF93BF93B9
:1035C0008091FE039091FF03A0910004B09101044B
:1035D000309102040196A11DB11D232F2D5F2D37BF
:1035E00020F02D570196A11DB11D20930204809358
:1035F000FE039093FF03A0930004B0930104809115
:10360000FA039091FB03A091FC03B091FD03019696
:10361000A11DB11D8093FA039093FB03A093FC03BB
:10362000B093FD03BF91AF919F918F913F912F91E7
:103630000F900FBE0F901F9018958FB7F8942091A0
:10364000FE033091FF0340910004509101048FBFAD
:10365000B901CA0108959FB7F8942091FA033091F7
:10366000FB034091FC035091FD0386B5A89B06C067
:103670008F3F21F02F5F3F4F4F4F5F4F9FBF542F22
:10368000432F322F2227280F311D411D511D82E06B
:10369000220F331F441F551F8A95D1F7B901CA0164
:1036A0000895EF92FF920F931F93CF93DF937B01C7
:1036B0008C010E942B1BEB010EC00E942B1B6C1B6C
:1036C0007D0B685E7340C8F30894E108F1080109B6
:1036D0001109C851DC4FE114F1040105110569F726
:1036E000CDB7DEB7E6E00C94F720019739F0880FEC
:1036F000991F880F991F02970197F1F70895789401
:1037000084B5826084BD84B5816084BD85B58260E6
:1037100085BD85B5816085BDEEE6F0E08081816084
:103720008083E1E8F0E01082808182608083808184
:1037300081608083E0E8F0E0808181608083E1EB5C
:10374000F0E0808184608083E0EBF0E08081816044
:103750008083EAE7F0E080818460808380818260FA
:1037600080838081816080838081806880831092E3
:10377000C1000895CF93DF93482F50E0CA018656C9
:103780009F4FFC0134914A575F4FFA01849188237F
:1037900069F190E0880F991FFC01E859FF4FA5914E
:1037A000B491FC01EE58FF4FC591D491662351F4BA
:1037B0002FB7F8948C91932F909589238C938881BF
:1037C00089230BC0623061F42FB7F8948C91932F4A
:1037D000909589238C938881832B88832FBF06C083
:1037E0009FB7F8948C91832B8C939FBFDF91CF91DF
:1037F0000895833071F0843028F48130A1F0823054
:1038000021F514C08630B1F08730D1F08430E9F46E
:1038100004C0809180008F7703C0809180008F7DED
:1038200080938000089584B58F7702C084B58F7D22
:1038300084BD08958091B0008F778093B000089583
:103840008091B0008F7D8093B0000895FF920F9318
:103850001F93F62E482F50E0CA0182559F4FFC015E
:103860002491CA0186569F4FFC0114914A575F4F1D
:10387000FA0104910023C9F0222319F0822F0E943B
:10388000F91BE02FF0E0EE0FFF1FEE58FF4FA59160
:10389000B4919FB7F894FF2021F48C911095812367
:1038A00002C08C91812B8C939FBF1F910F91FF9031
:1038B00008950F931F93482F50E0CA0182559F4FE0
:1038C000FC012491CA0186569F4FFC0104914A577E
:1038D0005F4FFA011491112319F420E030E015C074
:1038E000222319F0822F0E94F91B812F90E0880F6C
:1038F000991F84589F4FFC01A591B4918C9120E0B1
:1039000030E0802311F021E030E0C9011F910F91D8
:103910000895982F8E3008F09E50977080918B02FA
:103920008295880F880F807C892B80937C00809102
:103930007A00806480937A0080917A0086FDFCCFC3
:103940002091780040917900942F80E030E0282B7E
:10395000392BC9010895A0E0B0E0E1EBFCE10C9443
:10396000D9207C016B018A01C0E0D0E00FC0D601F4
:103970006D916D01D701ED91FC910190F081E02DE9
:10398000C7010995C80FD91F015010400115110535
:1039900071F7CE01CDB7DEB7E8E00C94F520DC017D
:1039A000ED91FC910190F081E02D09950895EF9241
:1039B000FF920F931F938C016DE00E94CF1C7C013E
:1039C000C8016AE00E94CF1C9C012E0D3F1DC90159
:1039D0001F910F91FF90EF900895EF92FF920F9338
:1039E0001F937C010E94CF1C8C01C7010E94D71C31
:1039F0009C01200F311FC9011F910F91FF90EF9083
:103A00000895CF93DF93EC016115710519F420E05F
:103A100030E00FC0DB010D900020E9F71197A61BE5
:103A2000B70BE881F9810280F381E02DAD010995A2
:103A30009C01C901DF91CF9108954F925F927F92CF
:103A40008F929F92AF92BF92CF92DF92EF92FF92AE
:103A50000F931F93DF93CF93CDB7DEB7A1970FB628
:103A6000F894DEBF0FBECDBF2C01742ECB012230E7
:103A700008F42AE019A231E2C32ED12CCC0EDD1EAF
:103A8000822E9924AA24BB24672D752FA5019401A9
:103A90000E94922079018A01C801B701A501940111
:103AA0000E945F20472D461B0894C108D1084A3068
:103AB00010F4405D01C0495CF6014083E114F1045B
:103AC0000105110521F07E2C5F2DC801DDCFC2015B
:103AD000B6010E94011DA1960FB6F894DEBF0FBE7D
:103AE000CDBFCF91DF911F910F91FF90EF90DF90AD
:103AF000CF90BF90AF909F908F907F905F904F90AE
:103B00000895DC012115310541F4ED91FC910190FE
:103B1000F081E02D642F099508950E941D1D0895E0
:103B2000EF92FF920F931F939A017B0100E010E048
:103B3000B801A7010E94811D1F910F91FF90EF9086
:103B40000895EF92FF920F931F939A01E62EFF24A0
:103B500000E010E0B801A7010E94811D1F910F91A4
:103B6000FF90EF900895A0E0B0E0E9EBFDE10C9448
:103B7000D920EC016A017B012115310541F4E8816E
:103B8000F9810190F081E02D642F09951BC02A3046
:103B90003105B1F477FF13C06DE20E94CF1C8C0198
:103BA00044275527BA014C195D096E097F09CE01DA
:103BB0002AE00E941D1D9C01200F311F04C02AE035
:103BC0000E941D1D9C01C901CDB7DEB7E8E00C9431
:103BD000F520EF92FF920F931F937B019A0100272C
:103BE000F7FC0095102FB801A7010E94B31D1F918B
:103BF0000F91FF90EF900895EF92FF920F931F9314
:103C00007C010E94E91D8C01C7010E94D71C9C0108
:103C1000200F311FC9011F910F91FF90EF90089560
:103C20000E94011D0895EF92FF920F931F937C0154
:103C30000E94101E8C01C7010E94D71C9C01200FFE
:103C4000311FC9011F910F91FF90EF9008950895C2
:103C50001F920F920FB60F9211242F933F934F9301
:103C60008F939F93EF93FF938091C00082FD1DC0BF
:103C70004091C60020914304309144042F5F3F4F90
:103C80002F733070809145049091460428173907AE
:103C900071F0E0914304F0914404ED5FFB4F4083E9
:103CA000309344042093430402C08091C600FF91E6
:103CB000EF919F918F914F913F912F910F900FBE58
:103CC0000F901F9018951F920F920FB60F9211240C
:103CD0002F933F938F939F93EF93FF9320918704AC
:103CE000309188048091890490918A0428173907BB
:103CF00031F48091C1008F7D8093C10014C0E091A8
:103D00008904F0918A04E95BFB4F2081809189044A
:103D100090918A0401968F73907090938A04809397
:103D200089042093C600FF91EF919F918F913F915D
:103D30002F910F900FBE0F901F901895A0E0B0E04C
:103D4000E4EAFEE10C94D520FC011382128288EE95
:103D500093E0A0E0B0E084839583A683B78388EBEB
:103D600092E0918380837587648757874687318B7C
:103D7000208B138B028BF58AE48AD78AC68AB18E90
:103D8000A08E938E828E8F85848F8889858F898976
:103D9000868F8A89878F8B8980A32096ECE00C948C
:103DA000F120AF92BF92DF92EF92FF920F931F9399
:103DB000CF93DF93EC017A018B01DD24403081EE5B
:103DC000580780E0680780E0780711F0DD24D3947D
:103DD00091E0A92EB12CEC89FD89DD2069F0C501A7
:103DE00008A002C0880F991F0A94E2F7808360E060
:103DF00079E08DE390E005C0108260E874E88EE120
:103E000090E0A80197010E9492202150304040404C
:103E10005040569547953795279580E120303807D3
:103E200020F0DD2011F0DD24D6CFE889F989308338
:103E3000EA89FB89208319A2EE89FF89408121E06C
:103E400030E0C9010C8C02C0880F991F0A94E2F778
:103E5000482B4083EE89FF894081C9010D8C02C047
:103E6000880F991F0A94E2F7482B4083EE89FF8957
:103E70004081C9010E8C02C0880F991F0A94E2F795
:103E8000482B4083EE89FF8980810F8C02C0220F6E
:103E9000331F0A94E2F7209528232083DF91CF91E6
:103EA0001F910F91FF90EF90DF90BF90AF9008951A
:103EB000DC011C96ED91FC911D97E05CFF4F219178
:103EC000319180819181281B390B2F733070C9018A
:103ED00008958BE894E00E94581F892B11F00E94EE
:103EE000271E0895DC011C96ED91FC911D97E05C66
:103EF000FF4F20813181E054F040DF01AE5BBF4FC6
:103F00008D919C9111972817390719F42FEF3FEFE6
:103F100007C08D919C91E80FF91F8081282F30E018
:103F2000C9010895DC011C96ED91FC911D97E05CA0
:103F3000FF4F20813181E054F040DF01AE5BBF4F85
:103F40008D919C9111972817390719F42FEF3FEFA6
:103F500010C08D919C911197E80FF91F20818D91D0
:103F60009C91119701968F73907011969C938E93EC
:103F700030E0C9010895DC0191968C9191978823D6
:103F800039F05496ED91FC915597808186FFF9CFD9
:103F900091961C920895CF93DF93EC01EE85FF85F7
:103FA000E05CFF4F20813181E054F0402F5F3F4FB4
:103FB0002F733070DF01AE5BBF4F8D919C911197D5
:103FC00028173907D1F3E05CFF4F80819181E054DD
:103FD000F040E80FF91F6083EE85FF85E05CFF4F3E
:103FE00031832083EE89FF89208181E090E00F8C6E
:103FF00002C0880F991F0A94E2F7282B208381E0E2
:1040000089A3EC89FD8980818064808381E090E0D0
:10401000DF91CF9108958F929F92AF92BF92CF92EE
:10402000DF92EF92FF920F931F9300D000D00F9278
:10403000EDB7FEB7319684E0ADB7BEB711968C935D
:1040400083E0818387E0828385E0838381E08483CA
:104050008BE894E063E074E047E454E025EC30E062
:1040600004EC10E0B0ECEB2EF12CA1ECCA2ED12C1C
:10407000F2ECAF2EB12CE6EC8E2E912C0E949E1EFF
:104080000F900F900F900F900F901F910F91FF9036
:10409000EF90DF90CF90BF90AF909F908F9008955A
:1040A000CF93DF930E947F1B0E94F718C9E6DFE1E0
:1040B0000E9479122097E1F30E94691FF9CF629F55
:1040C000D001739FF001829FE00DF11D649FE00D10
:1040D000F11D929FF00D839FF00D749FF00D659F71
:1040E000F00D9927729FB00DE11DF91F639FB00D70
:1040F000E11DF91FBD01CF0111240895AA1BBB1BAF
:1041000051E107C0AA1FBB1FA617B70710F0A61BD7
:10411000B70B881F991F5A95A9F780959095BC01F8
:10412000CD010895A1E21A2EAA1BBB1BFD010DC0F3
:10413000AA1FBB1FEE1FFF1FA217B307E407F50757
:1041400020F0A21BB30BE40BF50B661F771F881F33
:10415000991F1A9469F760957095809590959B01C9
:10416000AC01BD01CF01089597FB092E05260ED0A5
:1041700057FD04D0D7DF0AD0001C38F45095409585
:10418000309521953F4F4F4F5F4F0895F6F790952B
:104190008095709561957F4F8F4F9F4F08952F9217
:1041A0003F924F925F926F927F928F929F92AF92C7
:1041B000BF92CF92DF92EF92FF920F931F93CF9314
:1041C000DF93CDB7DEB7CA1BDB0B0FB6F894DEBFAB
:1041D0000FBECDBF09942A88398848885F846E84D1
:1041E0007D848C849B84AA84B984C884DF80EE801B
:1041F000FD800C811B81AA81B981CE0FD11D0FB624
:10420000F894DEBF0FBECDBFED010895EE0FFF1F86
:0C4210000590F491E02D0994F894FFCF84
:10421C0054582074696D656F757421005761697409
:10422C00696E672062696E640A00476F7420706B58
:10423C00740A006461746120676F6F640A005258DD
:10424C002068616E67007363616E6E6572206D6FBE
:10425C006465004F70656E4C52536E672052582047
:10426C007374617274696E672000206F6E204857FA
:10427C002000454550524F4D2064617461206E6F93
:10428C00742076616C6964206F722062696E6420A0
:10429C006A756D70706572207365742C20666F7210
:1042AC0063696E672062696E640A005361766564A7
:1042BC002062696E64206461746120746F204545CE
:1042CC0050524F4D0A004920616D20736C61766528
:1042DC0000456E746572696E67206E6F726D616CED
:1042EC00206D6F6465000020012201260221022747
:1042FC000323032604260526052B06240725072859
:10430C000729072AC01200001A400AA1204EA50056
:10431C001B1E27522C23308025000005400AA120AB
:10432C004EA50020244EA52C2330004B0000064047
:10433C000AD0009D49007B289D492C233000E100C8
:10434C000005400A4501D7DC03B81E0EBF00232E22
:10435C0048E801008A400A6001555502AD1E200054
:10436C000023C88025000005400AA1204EA500208E
:10437C00244EA52C23300002000200020002000291
:10438C000002000200020002000200020002000211
:10439C000002000200028813409C0801091203135A
:1043AC000E0F0001020000001000000008002000A9
:1043BC0000010000020000000100000200070B0CCD
:1043CC001011150000000000CB1FAB1C581F921FD2
:0443DC00721FBB1F72
:107E00000F92CDB7DEB7112484B714BE81FFF1D035
:107E100082E08093C00088E18093C10086E0809377
:107E2000C20080E18093C4008EE0CDD088249924E4
:107E3000CC24C394F5E0DF2EE1E1EE2E73E0F72EC3
:107E4000B6D0082F813479F4B2D08983C2D0898129
:107E5000823811F481E005C0813811F485E001C059
:107E600083E09ED09AC0823411F484E103C085344B
:107E700019F485E0B6D091C0853561F498D0082F0B
:107E800010E095D090E0982E8824802A912A880CC2
:107E9000991C82C0863521F484E0A3D080E0E1CF34
:107EA000843609F04CC083D082D0A82E80D0B82E62
:107EB00000E011E07CD0F80181938F01AE16D1F77C
:107EC00088D0FB2DF53489F4E0E0F1E00BC0F9999E
:107ED000FECF92BC81BC0894811C911C819180BD15
:107EE000FA9AF99AEA1598F358C08B2D863409F05E
:107EF00054C0F401F7BEE89507B600FCFDCFF401CD
:107F0000A0E0B1E02C9130E011968C91119790E0B7
:107F1000982F8827822B932B12960C01C7BEE895C9
:107F20001124329681E0A038B80761F7F401D7BE7A
:107F3000E89507B600FCFDCFE7BEE8952EC0843774
:107F4000F1F435D034D0182F32D0B82E42D0FB2DDA
:107F5000F63421F4F40105914F010CC0FB2DF534EA
:107F600049F4F999FECF92BC81BC0894811C911C04
:107F7000F89A00B5802F14D0115049F70EC08537FC
:107F800039F427D08EE10CD085E90AD08FE069CF93
:107F9000813511F488E017D01CD080E101D050CF9A
:107FA0009091C00095FFFCCF8093C600089580910A
:107FB000C00087FFFCCF8091C00084FD01C0A89560
:107FC0008091C6000895E0E6F0E098E19083808318
:107FD0000895EDDF803219F088E0F5DFFFCF84E10E
:107FE000DFCF1F93182FE3DF1150E9F7F2DF1F9166
:0E7FF0000895282E80E0E7DFEE27FF27099492
:027FFE0001057B
:0400000300007E007B
:00000001FF
